:100000000C9480010C94B8010C94B8010C94B801C4
:100010000C94B8010C94B8010C94B8010C94B8017C
:100020000C94B8010C94B8010C94D31E0C94A51F29
:100030000C94B2190C94B8010C94B8010C94B8014A
:100040000C94B8010C94B8010C94B8010C94B8014C
:100050000C94B8010C943A1A0C94B8010C94B801A1
:100060000C94B8010C94B8010C94B8010C94B8012C
:100070000C94B8010C94B8010C94B8010C94B8011C
:100080000C94B8010C94B8010C94B8010C94B8010C
:100090000C94B8010C94B8010C94B8010C94B801FC
:1000A0000C94B8010C94B8010C94B8018604860431
:1000B000B204B2041A053805500650064305DC05A3
:1000C000ED05ED05BC16B216BF1607170B170B177B
:1000D00007170B170B17E0160B17EA16F4160B177A
:1000E0000B170B170B1707170B170B1707170B1708
:1000F000CD160B170B170417041704170417041752
:10010000041704170417041709170B17BC16AF16AA
:100110000B170B170B170B170B170B170B170B17CF
:100120000B170B1709170B170B1707170B170217CE
:1001300002170217021702170217021702170217F7
:100140000917122039203121392031218520A8209A
:100150003121FF200E215F006000610057005C002C
:100160005D005E00000059005A005B00580062000C
:100170000000630000001C0352006F006100640077
:100180006B006900740020004D006900630072007C
:100190006F000000220354006800650056006100F3
:1001A0006E0020004B006500790062006F00610066
:1001B00072006400730000000403090409023B009C
:1001C000020100A0FA090400000103010100092155
:1001D0001101000122400007058103080001090404
:1001E0000100010300000009211101000122B600F5
:1001F000070582032000011201000200000008AE82
:10020000FE468801000102000105010902A10185E5
:10021000020901A100050919012908150025019508
:1002200008750181020501093009311581257F9585
:10023000027508810609381581257F9501750881A9
:1002400006050C0A38021581257F9501750881067F
:10025000C0C005010980A101850319012AB7001555
:100260000126B700950175108100C0050C0901A198
:1002700001850419012AA002150126A00295017525
:10028000108100C005010906A1018506050719E0D6
:1002900029E7150025019508750181020507190058
:1002A00029EF1500250195F0750181020508190156
:1002B0002905950575019102950175039101C00508
:1002C000010906A101050719E029E7150025019597
:1002D000087501810295017508810105071900293A
:1002E000FF150026FF009506750881000508190115
:1002F0002905950575019102950175039101C000CD
:1003000011241FBECFEFDAE0DEBFCDBF04B603FE7F
:1003100018C08091830290918402A0918502B091CF
:1003200086028730904BA740B04B59F4109283025D
:10033000109284021092850210928602E0E0F8E3A7
:10034000099511E0A0E0B1E0E8ECF3E402C005900B
:100350000D92A438B107D9F722E0A4E8B1E001C0BA
:100360001D92A338B207E1F70E942C120C94E221EF
:100370000C940000CF93DF93EC010E942D0DBE0181
:1003800080E090E0DF91CF910C943807873A9D454B
:1003900051F4FB018281882339F081E090E00E94D2
:1003A000BA0180E0089581E0089581E008950C94F9
:1003B000C60108950C94D9011F93CF93DF9300D009
:1003C00000D01F92CDB7DEB749835A836B8330913B
:1003D000870189819A81311114C0662359F0222343
:1003E00049F00E948B08182F682F89819A810E94FA
:1003F000360803C00E946008182F69817A81812F16
:1004000004C00E948B0869817A810F900F900F9031
:100410000F900F90DF91CF911F910C94B10FFC01C1
:10042000262F408151816281738184810C94DC018B
:1004300081E00895CF93DF93EC0160E00E940F020A
:10044000BE01DF91CF910C94DA010C94F5100C945D
:10045000F11008950E94E0060E9429022FEF84E324
:100460009CE0215080409040E1F700C000000C94D7
:10047000601A0F931F93CF93DF938C0161E00E946A
:100480000F02EC01B8010E94D7018823F1F1B801F5
:10049000CE010E94FE178823C1F1B801CE010E944F
:1004A000C214882391F1B801CE010E945A17882303
:1004B00061F1F8018281882309F1CB358DE5D807F8
:1004C000C1F050F4C115FCE5DF0781F0CF3DDC45FC
:1004D000A9F40E94C70D19C0CC35EDE5DE0761F027
:1004E000CD35DD4559F40E94050D08C00E942A0251
:1004F0000CC00E940E0D02C00E94110DC801DF91B8
:10050000CF911F910F910C94D50180E0DF91CF9195
:100510001F910F9108950E9495190C94A4020E94B6
:10052000A7020C949B1908950C94930281E00895FE
:100530000C9496020895CF93C82F0E9494028C2F9A
:100540000E949802CF91089580E00C949B020E9433
:100550005A180C949B020E945A1890918601891790
:1005600021F0809386010C949B020895CF93DF9332
:10057000CDB7DEB72B970FB6F894DEBF0FBECDBF59
:100580004F83588769877A878B8761110E94510C46
:100590009E012F5F3F4F86E0F90111928A95E9F79E
:1005A00085E0FE013796D90101900D928A95E1F719
:1005B00089819A814C815D81452B31F09F3F31F4D7
:1005C00091E08F3F19F403C091E001C090E090FFEB
:1005D00009C049815A816B817C818D819E810E94F5
:1005E000720B05C0C9010E9418028111F2CF2B962F
:1005F0000FB6F894DEBF0FBECDBFDF91CF91089547
:10060000FC01808191810E94CD080895CF938823B9
:1006100009F4A9C0C82F8238C1F40E945A1881FD7C
:10062000A2C069E380910201909103010E945019D8
:100630000E94730C2FEF81EE94E021508040904097
:10064000E1F700C0000069E319C0833801F50E949A
:100650005A1880FD88C063E58091020190910301E2
:100660000E9450190E94730C2FEF81EE94E02150EC
:1006700080409040E1F700C0000063E580910201F6
:10068000909103010E945B19CF910C94730C8438F4
:10069000C1F40E945A1882FD66C067E4809102018D
:1006A000909103010E9450190E94730C2FEF81EE6C
:1006B00094E0215080409040E1F700C0000067E4E2
:1006C000DDCF8CEF8C0F813AF8F48C2F0E9411173C
:1006D000811149C06C2F80910201909103010E9409
:1006E000D018882349F06C2F80910201909103016A
:1006F0000E945B190E94730C6C2F809102019091F3
:1007000003010E945019C0CF80E28C0F883048F45A
:10071000C77081E001C0880FCA95EAF70E94340CC7
:10072000B3CFEBE5EC0FE33040F4F0E0E95BFE4FD4
:10073000808190E0CF910C948E18E8E5EC0FE731C2
:1007400050F4F0E0EE0FFF1FE75EFE4F80819181D5
:10075000CF910C94A418CD3E30F08C2F0E94B11292
:10076000CF910C948313CF910895882309F464C02A
:10077000823879F40E945A1881FF5EC069E3809143
:100780000201909103010E9450190E94730C69E3C9
:1007900010C08338B1F40E945A1880FF4DC063E541
:1007A00080910201909103010E9450190E94730CE4
:1007B00063E580910201909103010E945B190C9402
:1007C000730C843879F40E945A1882FF35C067E4AC
:1007D00080910201909103010E9450190E94730CB4
:1007E00067E4E7CF9CEF980F913A10F4682FE1CFC0
:1007F00090E2980F983050F4877091E001C0990F03
:100800008A95EAF7892F0E943A0CD9CF9BE5980F79
:10081000933020F480E090E00C948E1898E5980FC7
:10082000973120F480E090E00C94A4188D3E20F0E5
:100830000E940C130C94831308951F93CF93DF939E
:10084000182FEB010E940603209741F08FE99FE0EB
:100850000197F1F700C000002197F6CF812FDF91BB
:10086000CF911F910C94B503893319F060E070E0CB
:1008700002C060E570E00C941D04882321F00E9402
:10088000340C0C94730C0895882321F00E943A0CC8
:100890000C94730C0895CF92DF92EF92FF920F9316
:1008A0001F93CF93DF937C01D62FC72FFC011281BA
:1008B000058102950F700E942A0C8823B9F011233C
:1008C000A9F08C2F807F803421F080E28D0F88305A
:1008D00068F08091690282FD09C082E00E94D30C19
:1008E0000E942A0C91E0D82ED92601C0D12CCC2E02
:1008F000C2948FE0C8228C2D90E08C30910508F0D6
:10090000CFC1FC01EA5AFF4F0C9479218C2F807FD4
:10091000CF70882311F0C295C07F112399F0CC23AA
:1009200009F4AAC180E28D0F883010F0D11104C003
:100930008C2F0E94340C03C08C2F0E94440C0E9408
:10094000730C9AC18D2F0E94B503CC2309F4A8C162
:1009500080E28D0F883038F1DD2329F18C2F0E9441
:100960004A0C24C08C2F807FCF70803211F0C2954A
:10097000C07FDD2319F0D130A1F13DC08091690223
:1009800082FF17C0112349F0CC2329F08C2F0E943D
:10099000340C0E94730C80E070C180E00E94B503AB
:1009A000CC2309F47DC18C2F0E943A0C0E94730C59
:1009B00077C1112371F0002341F0013031F40E941E
:1009C000540C8C2B0E945C0C6BC10E94540C8C2B21
:1009D0001DC0002319F0013009F462C10E94690CA6
:1009E00025C0112321F0063008F05AC10EC0053091
:1009F00008F056C11BC0112361F0002331F0F7014C
:100A0000858180FF39C18F7085838C2F0E943D04C2
:100A100047C1002359F0D93309F03FC1FFEF07EE7A
:100A200013E0F15000401040E1F735C18C2F0E94D7
:100A3000440436C18C2F86958695837019F08130D9
:100A400061F02EC1112321F08D2F9C2F937002C0D5
:100A500080E090E00E948E182BC1112321F08D2F91
:100A60009C2F937002C080E090E00E94A41820C1E7
:100A70008D2F112319F00E94B11202C00E940C1395
:100A80000E94831315C18C2F837009F047C0111188
:100A90000BC12D2F229526952770220F220F6D2F27
:100AA0006F70862F90E0A0E0B0E0022E04C0880FA7
:100AB000991FAA1FBB1F0A94D2F7D4FF10C04FE0A2
:100AC00050E060E070E004C0440F551F661F771FC0
:100AD0002A95D2F7409550956095709503C040E0F7
:100AE00050E0BA01C695C695C3708A019B01082BD8
:100AF000192B2A2B3B2BC901B801C23049F058F4FD
:100B0000C13019F00E944C07CFC00E943A07CCC0F8
:100B10000E945E07C9C00E943807C6C0112319F0A1
:100B20008C2F817001C08695882309F4BDC02D2FBC
:100B3000229526952770220F220F6D2F6F70862F1A
:100B400090E0A0E0B0E0022E04C0880F991FAA1F19
:100B5000BB1F0A94D2F7D4FF10C04FE050E060E012
:100B600070E004C0440F551F661F771F2A95D2F707
:100B7000409550956095709503C040E050E0BA01F3
:100B8000C695C695C3708A019B01082B192B2A2B89
:100B90003B2BC901B801C23049F058F4C13019F0FB
:100BA0000E94110881C00E94FF077EC00E94230896
:100BB0007BC00E94720778C0CF70112339F08C2F50
:100BC0000E9498078D2F0E943D046EC08D2F0E94B9
:100BD00044048C2F0E94B90767C0D23F21F128F44A
:100BE000D03F41F0D13FC1F043C0D33F19F1D43FD2
:100BF00079F03EC0112341F0053008F051C08C2F30
:100C00008F710E94DE074CC0063008F049C0F7CF54
:100C10008091690282FF18C0112339F08C2F8F71E7
:100C20000E9498073DC01123C9F38C2F8F710E9439
:100C3000B90736C0112329F08C2F8F710E948307CA
:100C40002FC00E947E072CC0112349F0CF718C2F3A
:100C50000E94980763E08C2F0E94B80C21C081E0AD
:100C60000E94D30C0230E0F082E00E94D30C18C046
:100C7000112331F0002391F28D2F0E94060310C042
:100C8000002399F2D93349F41FEF27EE33E01150D6
:100C900020403040E1F700C000008D2F0E94B503D6
:100CA00088EF8C0D843020F40E945A180E949B0219
:100CB000DD20C9F00E94260C80FD15C0F7011282CC
:100CC0000E94200C0E949807C7010E9494060E946F
:100CD000200CDF91CF911F910F91FF90EF90DF904B
:100CE000CF900C94B907DF91CF911F910F91FF9096
:100CF000EF90DF90CF9008950F931F93CF93DF93E2
:100D0000EC01688179818A810E94D8088C010E9457
:100D100035080E942607B801CE010E944B04DF91DE
:100D2000CF911F910F910895CF93DF93EC0198819C
:100D300089812B813C81232B31F08F3F31F481E07D
:100D40009F3F19F403C081E001C080E080FD1DC019
:100D5000CE010E943902811110C00E942A0C882302
:100D6000A1F08A81882389F08091690282FD0DC0FB
:100D700082E0DF91CF910C94D30CCE010E947C06CF
:100D8000CE01DF91CF910C941A02DF91CF9108959B
:100D900080E090E00E948E1880E090E00E94A4180D
:100DA0000E94510C0E94730C0E94B4140C94831383
:100DB00080910201909103010E9466190C94C8066B
:100DC0000E94410C0C94D80692959F70963079F051
:100DD00010F4925001C09A50923068F4803F69F04C
:100DE00018F4883E40F409C0843F29F406C0883EC8
:100DF00020F0813F11F080E0089581E00895FC012A
:100E0000808191810E94CD080E94E4060895CF93CD
:100E1000DF9300D000D01F92CDB7DEB70F900F90B8
:100E20000F900F900F90DF91CF910895CF93DF93A4
:100E300000D000D000D0CDB7DEB726960FB6F8941C
:100E4000DEBF0FBECDBFDF91CF9108950895089505
:100E50000C9427070C9428070E942A076093960198
:100E60007093970180939801909399010C94C80610
:100E70000C942C070F931F930091960110919701EA
:100E80002091980130919901602B712B822B932B2B
:100E90001F910F910C942C070F931F9300919601B3
:100EA000109197012091980130919901602371234D
:100EB000822393231F910F910C942C070F931F9360
:100EC000009196011091970120919801309199011C
:100ED00060277127822793271F910F910C942C076D
:100EE0000C9427070E9470076093920170939301FE
:100EF00080939401909395010C94C80660E070E093
:100F0000CB010C9472070F931F9341E050E060E017
:100F100070E08A019B0104C0000F111F221F331FC4
:100F20008A95D2F7C901B8011F910F910C947207ED
:100F30000F931F9341E050E060E070E004C0440F65
:100F4000551F661F771F8A95D2F780919201909165
:100F50009301A0919401B09195018A019B01082B06
:100F6000192B2A2B3B2BC901B8011F910F910C940F
:100F700072070F931F9341E050E060E070E004C0FF
:100F8000440F551F661F771F8A95D2F740955095DD
:100F9000609570958091920190919301A091940138
:100FA000B09195018A019B01082319232A233B2331
:100FB000C901B8011F910F910C9472070F931F93F1
:100FC00041E050E060E070E004C0440F551F661F30
:100FD000771F8A95D2F78091920190919301A09109
:100FE0009401B09195018A019B01082719272A27AE
:100FF0003B27C901B8011F910F910C9472070F9301
:101000001F930091920110919301209194013091CE
:101010009501602B712B822B932B1F910F910C94B8
:1010200072070F931F9300919201109193012091E9
:1010300094013091950160237123822393231F91A2
:101040000F910C9472070F931F93009192011091CE
:101050009301209194013091950160277127822797
:1010600093271F910F910C9472070895990F990F70
:10107000890FE82FE695E695E695877051E001C067
:10108000550F8A95EAF785E0E89FF0011124E857AB
:10109000FE4F20E030E070E04081CB01022E02C024
:1010A000969587950A94E2F7817081958427852328
:1010B000842781932F5F3F4F2530310569F70895CD
:1010C000990F990F890F682F669566956695982FE9
:1010D000977085E0689FB001112440E050E080E007
:1010E000FB01E40FF51FE857FE4F208130E0092E89
:1010F00002C0369527950A94E2F721703327042E13
:1011000001C0220F0A94EAF7822B4F5F5F4F4530F0
:10111000510531F70895BF92CF92DF92EF92FF927F
:101120000F931F93CF93DF938C01C0909201D090C7
:101130009301E0909401F090950180919601909137
:101140009701A0919801B0919901C82AD92AEA2A59
:10115000FB2ACFE1D0E0D701C6010C2E04C0B69522
:10116000A795979587950A94D2F780FD04C021979B
:1011700090F7B12C07C0BC2EB8018C2F0E94C50F70
:101180000197A9F38B2DDF91CF911F910F91FF90C4
:10119000EF90DF90CF90BF900895CF93DF93EC0155
:1011A0000E948B08BE010E94C50FDF91CF91089568
:1011B0001F93CF93DF93EB0190918701992321F047
:1011C000CB010E94CD0813C0882349F0CB010E94B7
:1011D0008B08182F682FCE010E94360804C0CB015F
:1011E0000E946008182FBE01812F0E94C50FDF9159
:1011F000CF911F9108951F93CF93DF93C0919A01D0
:1012000016E080919B01C81799F0D0E01C9FF00177
:101210001D9FF00D1124E456FE4F408151816281E3
:101220007381848195810E9416072196C770E9CF4A
:10123000DF91CF911F9108954091CC015091CD0144
:101240006091CE017091CF018091D0019091D10138
:101250000C941607EF92FF920F931F93CF93DF9397
:101260008091D10182958F7009F065C08091CE0187
:10127000882309F460C080919A01F0909B0110913D
:10128000CC010091CD016091CF017091D00191E02E
:101290001F3F09F090E0C0910001D0910101292F7A
:1012A00096E0E92E8F1509F446C06115710521F00D
:1012B0000F3F21F030E003C031E001C0322F90E059
:1012C00030FD36C0E89EF001E99EF00D1124DF01EB
:1012D000A456BE4F11963C911197301329C03C91F2
:1012E000311326C012963C911297311121C01396EA
:1012F0004D915C911497461B570B4C175D07C0F43A
:101300008091D1018F7080618093D101EF55FE4FA4
:1013100080818F70806180838CEC91E00E949406C4
:10132000DF91CF911F910F91FF90EF900C94FB08EC
:1013300001968770B7CFDF91CF911F910F91FF90EA
:10134000EF9008959F92AF92BF92CF92DF92EF926B
:10135000FF920F931F93CF93DF93CDB7DEB76197C3
:101360000FB6F894DEBF0FBECDBF8C0185E0F8014B
:10137000DE011D9601900D928A95E1F7D801129633
:10138000EC909091CC01E091CD012091CF01309172
:10139000D0012115310531F0EF3F31F481E09F3F5D
:1013A00019F403C081E001C080E0B82FB1709B2E1A
:1013B00080FD47C1D8014C9111965C91119713960D
:1013C000AD90BC9014978CECC82E81E0D82EF09094
:1013D000CE01B501621B730B209100013091010118
:1013E000FF2009F4D9C08091D1016217730708F07A
:1013F00095C0282F207F09F052C05E1313C04913F7
:1014000011C0FE2CE1100EC08F7080618093D1015D
:101410000E941C09C6010E9494068091D101F80126
:1014200085834DC1AB2831F05F3F31F481E04F3F00
:1014300019F403C081E001C080E080FD03C081E0B9
:101440008E2502C080E090E0F82FF170FF2E80FF23
:101450001CC080919A0120919B0136E0821709F40B
:101460000BC190E0389FF001399FF00D1124E45634
:10147000FE4F6181561306C06081461303C062812E
:10148000E61203C001968770E9CFFE2CEE2009F426
:1014900016C18091D10181608093D10154C05E1347
:1014A00006C0491304C0E11002C0F80199C0C80188
:1014B0000E94FF06882361F1EE2051F12091D101B5
:1014C000822F82958F7090E0029774F08091CC010A
:1014D0009091CD0198878F831986BB86AA862C8729
:1014E000CE0107960E94940686E0F801ACECB1E0CC
:1014F00001900D928A95E1F70E942A090E941C0929
:101500000AC05E1711F1C8010E94FF0681112CC0AC
:10151000C8010E949406FF24F394D1C0282F207F95
:1015200081F77A2DB98AA88A6E2D89890E940707CA
:101530008CEC91E00E94940686E0D6011D928A957B
:10154000E9F70E941C09F12CBAC04913DCCFE11065
:10155000DACFF8018583C8010E94940686E0D6019F
:101560001D928A95E9F7ABC0EE2091F22091D1014E
:10157000822F82958F7090E002970CF4B5CF809106
:10158000CC019091CD019A8389831B82BD82AC826C
:101590002E83CE010196A6CF6217730708F044C0D0
:1015A000FE2CEE2009F4B4CF5E1330C049132EC0D8
:1015B0002091D10120FD21C0822F82958F70482F6C
:1015C00050E041155105C9F0F80125834F30510510
:1015D00041F08F5F982F9295907F822F8F70892B8B
:1015E0008583C8010E94940686E0F801ACECB1E066
:1015F00001900D928A95E1F73CC086E0F801ACECD1
:10160000B1E001900D928A95E1F759C0C8010E949E
:10161000FF06811169CF8091D10181608093D10152
:10162000C8010E9494064BC07A2DB98AA88A6E2DF3
:1016300089890E94070786E0D6011D928A95E9F7FD
:1016400018C0EE2009F464CFC8010E94FF06F82EEE
:10165000882309F45DCF86E0F801ACECB1E001909D
:101660000D928A95E1F78CEC91E00E9400030E94B4
:101670002A090E941C0923C04D875E878D859E859F
:101680000E94CD08292F22952F70223028F49F70B8
:1016900039F0811105C00BC0243028F49F7049F443
:1016A000805E883020F0C8010E9494069F2CF92C9F
:1016B00006C0D80115969C91907F91F7F8CF8F2D99
:1016C00061960FB6F894DEBF0FBECDBFDF91CF910C
:1016D0001F910F91FF90EF90DF90CF90BF90AF9050
:1016E0009F9008951F93CF93DF93CDB7DEB72C97CC
:1016F0000FB6F894DEBF0FBECDBF4F835887698702
:101700007A878B879C87CE0107960E94A20988233F
:10171000D1F09F8188852A853B85232B31F08F3F2F
:1017200031F481E09F3F19F403C081E001C080E003
:1017300080FD47C04F81588569857A858B859C855A
:101740000E9416073EC086E0FE013796DE01119624
:1017500001900D928A95E1F7FF81E8856A857B8586
:101760006115710531F0EF3F31F481E0FF3F19F46D
:1017700003C081E001C080E080FD23C020919B0177
:1017800030E0C90101968770992740919A0150E095
:1017900084179507F1F1F983EA837D836C8396E0E2
:1017A000929FD001939FB00D1124A456BE4FFE010D
:1017B000319601900D929A95E1F780939B010E94DA
:1017C000FB0816E080919A0190919B01891771F1B5
:1017D000189FC001112484569E4F0E94A20988239D
:1017E00029F1E0919A011E9FF0011124E456FE4F69
:1017F0004081518162817381848195810E941607A5
:1018000080919A0190E001968770992780939A01C0
:10181000D9CF0E94E00610929B0110929A01ECEC45
:10182000F1E086E0DF011D928A95E9F72C960FB66C
:10183000F894DEBF0FBECDBFDF91CF911F91089509
:101840008091F20185958595859508958091F201A5
:10185000877008959091F201977081E009F480E01B
:10186000089580911502089590911502892B809317
:101870001502089580959091150289238093150291
:10188000089510921502089590911402892B809367
:101890001402089580959091140289238093140274
:1018A00008951092140208958091F3010895089507
:1018B0000C94570C0C94580C9091690292FD08C03E
:1018C0009091F301981721F08093F3010C945A0C36
:1018D00008958091F301882329F01092F30180E0AC
:1018E0000C945A0C0895CF93DF93E0910201F0918C
:1018F0000301809115028083E0910201F0910301C0
:10190000908180911402892B80838091F301882338
:1019100081F0E0910201F09103019081892B808395
:1019200080910201909103010E94BA1881110E94D6
:10193000690CC0910201D091030140E250E062EDD8
:1019400071E0CE010E949321892B69F080E2FE01B3
:10195000A2EDB1E001900D928A95E1F7CE01DF9101
:10196000CF910C946618DF91CF9108950C94570C89
:101970009091690292FD10C098E0899F9001112416
:10198000262B2093F2010E9498078091F201859501
:10199000859585950C94B60C0C9498071092F201DD
:1019A00080E00C94B60C2091F20180958223809304
:1019B000F201982F977099F430E0482F082E000C10
:1019C000550B2417350759F09091690292FD07C015
:1019D0008595859585950E94B9070C94CE0C089540
:1019E0009091690292FB222720F9281769F080FB69
:1019F00092F99093690280916802909169020E9425
:101A0000430D82E00C94D30C08958091690282FB0F
:101A1000882780F991E089270C94F00C81E00C94E0
:101A2000F00C80E00C94F00C6FEF7FEF80E090E022
:101A30000C94CC2180E090E00E94A82121E0893E16
:101A40009E4F09F020E0822F089582E090E00C94F0
:101A5000A02183E090E00C94A021682F83E090E027
:101A60000C94AE21CF9384E090E00E94A021C82F77
:101A700082E290E00E94A0212C2F30E0A901582B97
:101A8000CA01CF910895CF93C92F682F84E090E0C9
:101A90000E94AE216C2F82E290E0CF910C94AE2197
:101AA000AB01BC018FE090E00C94C021AB01BC0104
:101AB00083E190E00C94C02160E070E0CB010C94D5
:101AC000560D60E070E0CB010E94500D0C945C0D4F
:101AD00069EE7EEF80E090E00E94CC2160E082E041
:101AE00090E00E94AE2160E083E090E00E94AE2191
:101AF00010929601109297011092980110929901FC
:101B000060E084E090E00E94AE2160E082E290E03C
:101B10000E94AE2160E085E090E00E94AE2160E08E
:101B200086E090E00E94AE216FEF87E090E00E9497
:101B3000AE2140E050E0BA0188E090E00E94C02170
:101B400060E08DE090E00E94AE2140E050E0BA01FC
:101B500088E190E00E94C02160E087E190E00E946F
:101B6000AE2140E050E0BA018CE190E00E94C0213B
:101B700060E070E080E290E00E94CC2140E050E024
:101B8000BA0188E190E00E94C0210C94610D0C9490
:101B9000680D682F8EE090E00C94AE210E941F1A11
:101BA00060931E0270931F02809320029093210283
:101BB00060931A0270931B0280931C0290931D0283
:101BC000089585B7806885BF85B7806885BF08950B
:101BD00081E008950C94E80D08950C94EC0D0C949C
:101BE000EC0D0C94EF0D0C94EC0D0C94F30D0C9487
:101BF000EC0D0E94E10D81EA90E10E9450180E94D4
:101C0000F70D0C94F50D0E94ED0D0C94EC0D0E9457
:101C1000BB100C949A020E940A1A0E9492110E9410
:101C2000070E0C94F10D8F929F92AF92BF92CF92BC
:101C3000DF92EF92FF920F931F93CF93DF93CDB775
:101C4000DEB72A970FB6F894DEBF0FBECDBF0E9455
:101C5000A711982E81110E94CE0D86E1A82E82E058
:101C6000B82E00E010E0802E802F0E94DF10D82ECA
:101C7000F501C1905F01C826B1F40F5F1F4F04301A
:101C8000110589F78FEF89838A831B820E94131ABB
:101C90008160782F9D838C8349815A816B818D81EE
:101CA0000E94B6022FC08091220281FD0E94E510A1
:101CB000E12CFF24F3948C2D8F21F1F00E94EA0D8A
:101CC000882399F0EE828F82DF2081E009F480E0A2
:101CD00088870E94131A8160782F9A8789874E819E
:101CE0005F8168858A850E94B602F801EA5EFD4F31
:101CF0008081F826F08206C0E394FF0CF4E0EF1236
:101D0000DACFBBCF81E0911001C080E02A960FB6F8
:101D1000F894DEBF0FBECDBFDF91CF911F910F9121
:101D2000FF90EF90DF90CF90BF90AF909F908F90FB
:101D300008950E94130E0E94A1130C94AB02CF933E
:101D4000DF930E94CA0FEC01811521E5920708F08C
:101D500045C0811530E5930708F094C0883E910591
:101D600028F5803E910508F0F8C0883A910570F496
:101D7000853A910508F07CC08130910509F475C061
:101D800008F4E8C0049708F0E8C0E4C08F3B910570
:101D900008F0E0C0C85AD0E0CC0FDD1FC65BDE4FB4
:101DA0000990D881C02DCE019464D8C0811540E23D
:101DB000940758F4811551E0950708F0CEC08D3E88
:101DC000910508F4C7C09065C9C0C11580E4D80763
:101DD00008F4C0C0DF70CE01906AC0C0811525E54F
:101DE0009207A8F4811534E5930708F095C0811592
:101DF00043E5940708F07BC0811552E5950708F08C
:101E000061C0D82FCC27CE01816F906AA7C0C115C1
:101E100089E5D807A0F4C11528E5D20708F082C0EB
:101E2000C11536E5D30708F095C08C2F0E945E10CF
:101E30008F7190E0D82FCC27CE0190628FC0C11552
:101E40004AE5D40708F474C0CE019056811590423B
:101E500008F080C08D2F8F710E945E10DD27D06248
:101E60008F71AE01582BCA0179C081E090E076C035
:101E7000C55AD0E0C858DE4F8881C82FD0E0CE01C7
:101E800090646CC074E0969587957A95E1F7282F59
:101E900023703C2F337081E090E002C0880F991FBF
:101EA0003A95E2F79C68AC01522B9A019C2F9F70E7
:101EB0009695969550E2959FE0011124C9018C2BCF
:101EC0009D2B4CC08370992721E030E002C0220F87
:101ED000331F8A95E2F79C2F9695969580E2989FFE
:101EE000E0011124C22BD32BCE019C6837C0837034
:101EF000992721E030E002C0220F331F8A95E2F7D4
:101F00009C2F9695969540E2949FE0011124C22B58
:101F1000D32BCE019A6822C0D82FCC27CE01846F54
:101F2000906A1CC0DC2FCC27CE01806F906A16C04F
:101F30008C2F8F700E945E1094E0D695C7959A956D
:101F4000E1F7CF70D0E0DC2FCC27D0699E01282BA1
:101F5000C90104C080E090E001C0CE01DF91CF91C3
:101F60000895E72FF0E094E0899FE00DF11D112422
:101F7000EE0FFF1FEE0FFF1FE60FF11DEE0FFF1F0D
:101F8000EA5AFE4F8591949108950E94B10F0E94E4
:101F90009F0E08958238910569F1B0F4813391055F
:101FA00009F46DC048F48932910509F463C08A329E
:101FB000910509F469C008958533910509F455C068
:101FC00089339105B9F00895833E910569F138F49C
:101FD000803E9105B1F0823E910509F10895863E5B
:101FE0009105A9F1873E9105B9F1843E910509F06B
:101FF00064C023C02091680220FD4FC021FD4DC068
:1020000008958091680280FD44C08091690280FF3C
:1020100044C08091680284FD42C083EE4DC080912F
:10202000680282FF38C0F5CF8091680282FD33C01C
:102030008091690280FD31C0ECCF8091690281FFFF
:1020400032C08091680284FD2AC087EE35C080913D
:10205000680283FF26C0F5CF8091680283FD21C00E
:102060008091690281FD1FC0ECCF8091680285FDDF
:102070001CC01DC08091680285FD19C016C08091EA
:10208000680286FD16C017C08091680286FD13C0E5
:1020900010C089E311C082EE0FC080EE0DC080E059
:1020A0000BC086EE09C084EE07C089E205C085E357
:1020B00003C08AE201C081E390E008959091680234
:1020C00092FF0DC0282F2871283019F4877F846073
:1020D00006C0282F2471243011F48B7F886093FF71
:1020E0000DC0282F2871283119F4877E846106C01D
:1020F000282F2471243111F48B7E8861209169028C
:1021000020FF0DC0382F3871383019F4877F816077
:1021100006C0382F3171313011F48E7F886021FF75
:102120000DC0282F2871283119F4877E816106C0DF
:10213000282F2171213111F48E7E886194FD877ED4
:10214000089580E008950C94140D0E94A7118FE368
:102150009CE90197F1F700C000000E94A71180E000
:102160000E94DF1080FF04C00E94A3100C94601A2C
:1021700008950C94A5100E941A0D811102C00E94AE
:10218000C70D0E94250D809322020E94320D90936C
:102190006902809368020E94B9100E94290D682F7D
:1021A00070E080E090E00E943807609192017091A9
:1021B000930180919401909195010C947007E82F00
:1021C000F0E0E259FD4F80810895089580EA8A95F4
:1021D000F1F7089500C008950C94E61008950C944A
:1021E000EE100C94EF100C94EE100C94F310F89485
:1021F000E82FE295EF70F0E031A1282F2F7081E0F9
:1022000090E001C0880F2A95EAF7982F90959323C4
:1022100091A392A1892B82A3789408950F931F9381
:10222000CF93DF93CFE7D1E089918F3F11F00E94E8
:10223000F71081E0C338D807B9F7CBE7D1E00FE753
:1022400011E089918F3F11F00E94F7100C171D07C4
:10225000C1F7DF91CF911F910F910895CF92DF9237
:10226000EF92FF920F931F93CF93DF938C01C62FB2
:10227000D0E0CE0181589E4F7C01FC0190819F3FB0
:1022800009F447C0D62EF894E92FE295EF70F0E0FC
:1022900081A19F7021E030E001C0220F9A95EAF7FA
:1022A000822B81A382A12095282322A378940E94C7
:1022B000EA10EBE7F1E04FE751E031E0C12C21916A
:1022C0002F3F89F0A22FA295AF70B0E090968C912D
:1022D00090E02F7002C0959587952A95E2F780FDD2
:1022E00002C0832F01C080E0C82A330F4E175F075A
:1022F00031F7F70180818F3F11F00E94F71061E004
:10230000C11001C060E08D2D0E94EC10C00FD11FE4
:10231000C882DF91CF911F910F91FF90EF90DF90D6
:10232000CF9008950E940E1184E0EEE6F2E0DF0106
:10233000982F1D929A95E9F7EAE6F2E0DF011D92E7
:102340008A95E9F784E00E94E9110C9425021F9315
:10235000CF93DF9300D000D0CDB7DEB719821A82B9
:102360001B821C8210E0612FCE0101960E942E116B
:102370001F5F1430C1F744E050E0BE016F5F7F4F34
:102380008AE692E00E94932111E0009709F410E0A0
:10239000892B61F089819A81AB81BC8180936A022B
:1023A00090936B02A0936C02B0936D02212F44E0D6
:1023B0006EE672E08AE692E00E94EA110E9427022D
:1023C000812F0F900F900F900F90DF91CF911F9161
:1023D00008950895FF920F931F93CF93DF938C017D
:1023E000F62ED72FC42F222349F081E080932502B7
:1023F0000E94131A90932402809323028091250255
:102400008823C1F080912302909124020E942B1A0C
:10241000059780F0EF2DFD2FD8014C2F50E0CD0116
:10242000801B910B841795071CF48D918193F7CF36
:1024300010922502DF91CF911F910F91FF90089587
:102440000E942B1C0E940B0E0C94371C0E943B1CFC
:102450000E94990E0C94551C0E94B1190E94121CE6
:102460000E94F90D0E9420120E9426120E94030E63
:10247000FBCF80912C0280FF06C06091090170E0C3
:10248000660F771F26C081FF04C06091090184E0B8
:1024900005C082FF07C06091090188E0689FB00114
:1024A000112417C090912B029923D1F0609108015B
:1024B000961788F72091090188E0289F9001112440
:1024C000929FA001939F500D112470E0CA010E94B9
:1024D00065216038710540F46115710519F406C075
:1024E00068E070E0862F08958FE7089581E00895F1
:1024F00080912C0280FF08C06091050170E0759505
:1025000067957595679521C081FF06C060910501AB
:1025100070E07595679519C082FF04C06091050150
:1025200070E010C090912A02992399F06091040103
:102530009617A0F780910501899FC001112470E0D2
:102540000E9465216038710540F46115710519F428
:1025500006C061E070E0862F08958FE7089581E05E
:1025600008958D3E21F40E943912819504C08E3E5B
:1025700029F40E9439128093300208958F3E21F48D
:102580000E943912819504C0803F29F40E943912BB
:1025900080932F020895893F19F40E94781205C094
:1025A0008A3F31F40E947812819580933102089518
:1025B0008B3F21F40E947812819504C08C3F29F44E
:1025C0000E9478128093320208959FE0980F98300D
:1025D00078F421E030E0A90102C0440F551F9A951C
:1025E000E2F7CA0190912E02892B80932E02089562
:1025F0008D3F21F480912C0281600BC08E3F21F42D
:1026000080912C02826005C08F3F29F480912C02BA
:10261000846080932C0208958D3E39F490913002AD
:1026200097FF35C01092300259C08E3E29F4909128
:1026300030021916BCF32BC090912F028F3E29F463
:1026400097FF25C010922F0249C0803F19F4191638
:10265000CCF31DC090913102893F29F41916BCF4C6
:10266000109231023BC08A3F19F497FF10C0F8CF97
:102670008B3F39F49091320297FF09C010923202D9
:102680002DC08C3F21F4909132021916BCF39FE0CB
:10269000980F983080F421E030E0A90102C0440F87
:1026A000551F9A95E2F7CA01809590912E028923D1
:1026B00080932E0213C08D3F21F480912C028E7FD7
:1026C0000BC08E3F21F480912C028D7F05C08F3F7F
:1026D00029F480912C028B7F80932C0280912F0211
:1026E000811106C080913002811102C010922B022C
:1026F00080913102811106C080913202811102C0A5
:1027000010922A0208950E94131A20912F0221117B
:1027100004C020913002222321F09093290280935B
:10272000280220913102211104C02091320222237B
:1027300021F090932702809326028DE292E00C9480
:102740008018EF92FF920F931F93CF93DF9300D0E7
:1027500000D000D0CDB7DEB786E0EDE2F2E0DE01DA
:10276000119601900D928A95E1F7E0902F02F0907A
:102770003002009131021091320210922F02109219
:1027800030021092310210923202E11003C0FF2099
:1027900009F45DC080912802909129020E942B1AB1
:1027A000AC0190912B02992339F020910A0130E07D
:1027B0002417350758F04BC020910B018AE0289F61
:1027C000900111242417350718F041C09F3F19F0DC
:1027D0009F5F90932B02EE2061F00E9439121E142D
:1027E00014F09FEF01C091E0989F902D11249093D9
:1027F0002F02FF2061F00E9439121F1414F09FEF86
:1028000001C091E0989F902D112490933002309157
:102810002F023323E1F0209130022223C1F045EB57
:102820003403C0011124992319F090932F0203C09F
:1028300081E080932F0235EB2303C00111249923FB
:1028400019F09093300203C081E0809330020111AF
:1028500003C0112309F45DC08091260290912702E4
:102860000E942B1AAC0190912A02992339F02091F1
:10287000060130E02417350758F04BC020910701BE
:102880008AE0289F900111242417350718F041C0D1
:102890009F3F19F09F5F90932A02002361F00E94EE
:1028A0007812101614F09FEF01C091E0989F902DC0
:1028B000112490933102112361F00E9478121116B5
:1028C00014F09FEF01C091E0989F902D11249093F8
:1028D0003202309131023323E1F02091320222237F
:1028E000C1F045EB3403C0011124992319F09093F2
:1028F000310203C081E08093310235EB2303C00134
:102900001124992319F09093320203C081E080933F
:10291000320280912F0281110BC08091300281110F
:1029200007C080913102811103C080913202811170
:102930000E948313EB82FC820D831E8386E0FE01DE
:102940003196ADE2B2E001900D928A95E1F72696BC
:102950000FB6F894DEBF0FBECDBFDF91CF911F91B0
:102960000F91FF90EF900895EDE2F2E086E0DF0135
:102970001D928A95E9F710922B0210922A0210926A
:102980002C020895CF93DF93EC01FB018281882311
:1029900009F43CC1C430FDE5DF0760F4CB3F9CE5A2
:1029A000D90788F49E0122503C452431310508F0B6
:1029B0002EC109C0C236EDE5DE0729F0C63AFDE5B5
:1029C000DF0709F024C10E94320D909369028093C1
:1029D0006802C1318CE5D80709F4C6C008F042C0CE
:1029E000C930ECE5DE0709F49BC000F5C5308CE585
:1029F000D80709F485C078F4C330ECE5DE0709F4A4
:102A000078C008F07AC0C230DC4509F0F5C080918A
:102A100068028160EFC0C7309CE5D90709F478C02F
:102A200008F07AC0809168028061E4C0CD30FCE596
:102A3000DF0709F487C058F4CB309CE5D90709F4C7
:102A400079C008F07BC08091680288606FC0CF3089
:102A5000FCE5DF0709F480C008F082C080916802BD
:102A6000877FC8C0CE3F9CE5D90709F471C000F547
:102A7000C531FCE5DF0709F485C068F4C3319CE586
:102A8000D90709F475C008F095C00E94E00680914E
:102A900068028F77AFC0CC3FFCE5DF07A9F108F0F3
:102AA00054C0CB3FDC4509F0A7C08091690240C00B
:102AB000C230EDE5DE0709F489C058F4C1158DE593
:102AC000D80709F45AC008F069C080916902826091
:102AD0002FC0C236EDE5DE0709F47CC0C63AFDE53D
:102AE000DF0709F481C0C330DD4509F085C080E00F
:102AF0006EC08091680282607DC08091680216C0BD
:102B000080916802886076C08091690282604FC0BF
:102B10008091680280626EC08091680280646AC0A1
:102B20000E94E00680916802806864C0846062C090
:102B300081603DC0809168028E7F5CC08091680298
:102B40008D7F58C08091680216C08091690218C0BC
:102B5000809169028D7F2BC0809168028F7E4AC070
:102B6000809168028F7D46C0809168028F7B42C051
:102B700080916802877F8B7F3DC0809169028D7F45
:102B80008E7F15C08091680282FB222720F991E098
:102B9000922790FB82F990FB83F92CC08091690207
:102BA000982F909591708E7F892B90FB81F980935F
:102BB000690222C00E94E0068091680287FB2227FA
:102BC00020F991E0922790FB87F914C081E00E94E0
:102BD000C90D12C08091680284FB222720F991E080
:102BE000922790FB84F906C080916802982F9095F7
:102BF00090FB80F98093680280916802909169024D
:102C00000E94430D0E94E00680E001C081E0DF9158
:102C1000CF910895893289F1F0F4843171F1B0F4E3
:102C2000873009F077C081E080930B0184E18093C5
:102C30000A018AE0809309018EE18093080188E00F
:102C40008093050188E28093040164C092EE980F9E
:102C50009A30F0F05FC0803509F444C028F48F3416
:102C600009F058C08AE03FC0813529F0823509F06B
:102C700051C081E038C08FEF36C080913502882383
:102C800079F110923502109234021092330242C050
:102C90008D5180933502833099F038F4813069F09A
:102CA0008230D9F48AE091E00DC0853099F078F057
:102CB000863099F484E091E005C08BE091E002C099
:102CC00089E091E0909334028093330223C088E03E
:102CD00091E0F8CF85E091E0F5CF109235021AC06F
:102CE00080E0089586EFE0913302F091340230974E
:102CF00089F02081082E000C990B820F911D8F3FC7
:102D0000910519F014F08FEF04C097FF02C01082F4
:102D100001C0808381E008950F931F9341E050E04C
:102D200060E070E08A019B0104C0000F111F221FA8
:102D3000331F8A95D2F7C901B8010E9438071F9145
:102D40000F910C94E006482F50E0FA013597EF33CD
:102D5000F10508F060C0EE59FF4F0C9479210E94F4
:102D6000C70D55C080912202817F8E7F8093220201
:102D700081E08093360208950E942A0248C0809123
:102D80002202982F9095917090FB80F980932202F7
:102D900091113DC0897F877F10C08091220281FB05
:102DA000222720F991E0922790FB81F9809322025B
:102DB000992369F18091220281608093220227C0C9
:102DC0008091220282FB222720F991E0922790FB3A
:102DD00082F9ECCF8091220283FB222720F991E037
:102DE000922790FB83F9E2CF0E94E006809168026F
:102DF00087FB222720F991E0922790FB87F98093A7
:102E0000680205C0895301C08D510E948C1681E073
:102E1000089580E0FACF80E0089580E008950C9452
:102E20000D17CF93C82F80913602813069F038F0AA
:102E30008230C1F58C2F0E940A1681E039C00E94B1
:102E4000310C823289F504C00E94310C823261F467
:102E50008C2F0E940F17811104C08C2F0E94A31683
:102E60001FC081E090E01CC08C2F0E940D178111C3
:102E700016C0C43189F058F4CB3089F0C031B1F4B8
:102E800082E08093360288E30E940A1608C0C932A5
:102E900019F0C83321F00AC01092360207C081E051
:102EA000817006C01092360280E002C080E0F8CF48
:102EB000CF910895CF93DF9386319C4541F5EB0187
:102EC0000E94310C982F8A812091020130910301D8
:102ED000882379F09A7A81E009F480E080933702C0
:102EE000911102C069E201C065E3C9010E94501955
:102EF0000AC080913702811102C069E201C065E316
:102F0000C9010E945B190E94730C80E001C081E03E
:102F1000DF91CF9108950F931F93CF93DF93C42F29
:102F2000D22FFC0182818823C9F040933A020E948B
:102F3000131A909339028093380280E28C0F883004
:102F400008F057C0C77081E001C0880FCA95EAF742
:102F5000DF91CF911F910F910C943D0480913A0223
:102F6000481330C080913802909139020E942B1A88
:102F7000883C910538F510E21D0FCD17B9F080E2BD
:102F80008C0F883040F4C77081E001C0880FCA956B
:102F9000EAF70E944404183028F581E09D2F9770CD
:102FA00001C0880F9A95EAF70E943D04802F0E9485
:102FB00034041830F0F4D77081E001C0880FDA953E
:102FC000EAF70AC080E28C0F883098F4C77081E07D
:102FD00001C0880FCA95EAF7DF91CF911F910F9139
:102FE0000C944404802FDF91CF911F910F910C948A
:102FF0003404DF91CF911F910F9108950F939C019D
:10300000CB01243F4CE5340731F188F4293DFCE540
:103010003F07D9F02A3D4CE5340779F1283D3C457E
:10302000A9F506E221EE41EE68ED7CE52BC0263FD6
:10303000FCE53F07E1F0A8F0273F3C4539F507E202
:1030400025EE46EE67EF7CE51DC007E225EE45EE76
:1030500069ED7CE517C006E221EE40EE64EF7CE509
:1030600011C007E225EE44EE65EF7CE50BC006E2F9
:1030700021EE42EE66EF7CE505C008E221E045EE78
:103080006AED7CE50E948B1780E008C0FC0182811C
:10309000882319F010923A0201C081E00F9108953F
:1030A00090938501809384010895909340028093CA
:1030B0003F020895E0913F02F0914002309721F0E5
:1030C0000190F081E02D099480E00895E0913F02A5
:1030D000F0914002309799F020911801222359F085
:1030E0002091680227FF07C0DC012C9111962C93D8
:1030F000119726E02C930280F381E02D0994089526
:10310000E0913F02F0914002309739F022E0DC017B
:103110002C930480F581E02D0994089520913D02BF
:1031200030913E022817390771F090933E02809348
:103130003D02E0913F02F0914002309721F006807D
:10314000F781E02D0994089520913B0230913C02D3
:103150002817390771F090933C0280933B02E0916D
:103160003F02F0914002309721F00084F185E02D7C
:1031700009940895FC01329680911801882331F05A
:103180008091680287FF02C09EE101C096E080E066
:10319000915028F021912223D9F38F5FF9CF089520
:1031A000662351F1209118012223E9F02091680251
:1031B00027FF19C0462F4695469546954E31E0F4B7
:1031C000677021E030E002C0220F331F6A95E2F7FA
:1031D000FC01E40FF11D828190E02823392381E076
:1031E000232B69F409C0FC013296089621916217DD
:1031F00029F0E817F907D1F780E0089581E00895F4
:103200009C01FC0132969FEF80E04191461789F0C6
:103210009F3F19F4411101C0982F8F5F8630A9F7A5
:103220009F3F39F0F901E90FF11D97FDFA9562838F
:10323000089508959C012A5F3F4FFC014281461387
:1032400001C01282019682179307B9F70895262FBD
:103250002695269526952E3168F4FC01E20FF11D86
:10326000677021E030E001C0220F6A95EAF78281A1
:10327000282B22830895262F2695269526952E31D4
:1032800070F4FC01E20FF11D677021E030E001C035
:10329000220F6A95EAF720958281282322830895D8
:1032A00020911801222329F02091680227FD0C9417
:1032B00027190C94001920911801222329F020913C
:1032C000680227FD0C943B190C941A1920911801DF
:1032D000FC013296222331F08091680287FF02C000
:1032E0008EE101C086E0DF011D928A95E9F708951D
:1032F00008950C94781983E0809341020C94791915
:10330000811102C081E001C082E0809341020C94EF
:1033100079190C94801981E0809341020C947919F9
:103320000C948B1908950C9492190C9493190C9485
:1033300092190C9492190C949219CF930E94991996
:103340000E94A7110E949719C0E08C2F0E94DF10E5
:10335000811104C0CF5FC430C1F701C081E0CF91BB
:10336000089508951F920F920FB60F9211248F9314
:103370009F93AF93BF9380914202811113C08091BC
:10338000720290917302A0917402B09175024196FD
:10339000A11DB11D8093720290937302A0937402D9
:1033A000B0937502BF91AF919F918F910F900FBE17
:1033B0000F901F90189580917A02843031F10E940D
:1033C0008B021092420220E488E190E00FB6F8945C
:1033D000A895809360000FBE2093600083B7817F23
:1033E000846083BF83B7816083BF7894889583B7F7
:1033F0008E7F83BF0FB6F894A89580916000886196
:1034000080936000109260000FBE08950E94E00655
:103410000C948F0282E084BD93E095BD9AEF97BD36
:1034200080936E0008952FB7F89480917202909166
:103430007302A0917402B09175022FBF08952FB747
:10344000F89460917202709173028091740290916D
:1034500075022FBF08959C014FB7F89480917202B6
:1034600090917302A0917402B09175024FBF821BBC
:10347000930B089578941F920F920FB60F92112418
:103480008F939F93AF93BF93809172029091730239
:10349000A0917402B09175020196A11DB11D809397
:1034A000720290937302A0937402B0937502BF915D
:1034B000AF919F918F910F900FBE0F901F90189515
:1034C00081E08093E00080E28093D8001092C900F0
:1034D0008FE19EE40197F1F700C0000087E090EBD8
:1034E000DC018093830290938402A0938502B093C1
:1034F00086029CE088E10FB6F894A895809360005E
:103500000FBE90936000FFCF8091660208950895EA
:1035100022E02093E9002FEF3091E800215035FDA3
:1035200006C035ED3A95F1F700002111F5CF209155
:10353000E80025FF0BC040E050E066E070E00E942C
:10354000C71C8091E8008E778093E8000895CF93A0
:10355000DF9320911801222339F02091680227FF80
:1035600003C060E222E002C068E021E02093E900AD
:103570002FEF3091E800215035FD06C035ED3A952A
:10358000F1F700002111F5CF2091E80025FF1DC0C3
:10359000EC0180911801811105C040E050E068E025
:1035A00070E003C070E040E050E0CE010E94C71C14
:1035B0008091E8008E778093E80080E2FE01A6E427
:1035C000B2E001900D928A95E1F7DF91CF910895D5
:1035D00080934302709345026093440280917A0283
:1035E000843001F582E08093E9008FEF9091E8004C
:1035F000815095FD06C095ED9A95F1F70000811177
:10360000F5CF8091E80085FF0DC040E050E063E019
:1036100070E083E492E00E94C71C8091E8008E77FE
:103620008093E8000895BC0184E00C94E81ABC0182
:1036300083E00C94E81A80917902811109C00E94FC
:10364000581E0E94B51E8091E20084608093E200C3
:1036500008951092790208950C9490196091760261
:1036600081E0611101C080E00C947B1990917A0295
:1036700081E0943009F080E0609176020C9480192A
:1036800042E061EC81E00E94D11D42E261EC82E007
:103690000E94D11D90917A0281E0943009F080E07F
:1036A000609176020C94891980917C02833009F430
:1036B00061C030F4813071F0823009F49AC008950D
:1036C0008A3009F486C08B3009F46CC0893009F067
:1036D000A8C020C080917B02813A09F0A2C08091ED
:1036E000E800877F8093E80080917F0290918002BC
:1036F000892B21F460E286E492E003C060E080E080
:1037000090E070E00E94121D8091E8008B7780931A
:10371000E800089580917B02813209F082C0809197
:103720007F0290918002029708F07BC08091E800B0
:10373000877F8093E8008091E80082FD05C080913A
:103740007A028111F8CF6DC02091F3008091F200D0
:1037500090E0922B029731F48091F100813011F0CA
:10376000863021F48091F100809366028091E80018
:103770008B7753C080917B02813A09F052C08091CF
:103780007F0290918002892B09F04BC08091E80064
:10379000877F8093E8008091E80080FFFCCF8091D4
:1037A000180136C080917B028132D9F580917F0269
:1037B00090918002892BA9F58091E800877F809302
:1037C000E8000E94061E80917D02809318010C94EF
:1037D000E00680917B02813221F58091E800877FAD
:1037E0008093E8000E94061E80917E02809367020B
:1037F000089580917B02813AA1F48091E800877F4F
:103800008093E8008091E80080FFFCCF8091670200
:103810008093F1008091E8008E778093E8000C940B
:10382000061E089584B7877F84BF0FB6F894A895C5
:1038300080916000886180936000109260000FBEEC
:1038400090E080E80FB6F894809361009093610057
:103850000FBE0C948B190E94581E0E94B51EE2EEFA
:10386000F0E080818460808378940C944A218CE01D
:1038700091E00C94551880917A028530A9F48091DA
:103880007A02853079F40E94DB19809178028823CE
:10389000B1F30E949D19882391F30E94B11C0E94EC
:1038A000E006EDCF0C94061A089508950C94581C68
:1038B000292F332723303105C9F060F42130310539
:1038C00081F02230310509F044C08BE390E02CEB0D
:1038D00031E043C021323105E1F02232310549F1B6
:1038E00038C082E190E027EF31E037C0992781307E
:1038F000910549F028F0029761F5E6E7F1E005C08F
:10390000E8EBF1E002C0E4E9F1E0849190E09F018E
:1039100024C06115710541F061307105D1F489E071
:1039200090E027EE31E019C089E090E02EEC31E024
:1039300014C06115710541F06130710551F486EBD9
:1039400090E029E032E009C080E490E02FEB32E023
:1039500004C080E090E020E030E0FA013183208371
:10396000089580E189BD82E189BD09B400FEFDCFE3
:103970008091D8008F7D8093D8008091E000826094
:103980008093E0008091E00081FDFCCF0895CF920C
:10399000DF92EF92FF920F931F93CF93DF93EC018F
:1039A0008B017A010E94251E811133C0E114F104BC
:1039B00039F0F70180819181081B190BC80FD91FBD
:1039C000C12CD12C0115110519F18091E80085FD5C
:1039D00016C08091E8008E778093E800E114F1042E
:1039E00049F0F70180819181C80ED91ED182C08231
:1039F00085E00FC00E94251E882321F30AC089910B
:103A00008093F10001501109FFEFCF1ADF0ADACFDE
:103A100080E0DF91CF911F910F91FF90EF90DF90A9
:103A2000CF900895209181023091820226173707A6
:103A300048F06115710539F42091E8002E77209344
:103A4000E80001C0B901FC0120E06115710579F1C0
:103A500080917A028823F1F18530F1F18091E800BC
:103A600083FD3CC08091E80082FD2EC08091E8007B
:103A700080FFEBCF2091F3008091F20090E0922B39
:103A80006115710551F08830910538F4219120932A
:103A9000F100615071090196F3CF21E0089709F018
:103AA00020E08091E8008E778093E800CECF21114E
:103AB000CFCF0AC080917A02882361F0853061F00F
:103AC0008091E80083FD0AC08091E80082FFF2CF78
:103AD00080E0089582E0089583E0089581E00895EC
:103AE00020918102309182022617370748F0611534
:103AF000710539F42091E8002E772093E80001C089
:103B0000B901FC0120E06115710591F180917A0203
:103B1000882309F440C0853009F43FC08091E80053
:103B200083FD3DC08091E80082FD2FC08091E800B8
:103B300080FFE9CF2091F3008091F20090E0922B7A
:103B40006115710559F08830910540F42491209356
:103B5000F1003196615071090196F2CF21E008978A
:103B600009F020E08091E8008E778093E800CBCFC9
:103B70002111CCCF0AC080917A02882361F0853070
:103B800061F08091E80083FD0AC08091E80082FF27
:103B9000F2CF80E0089582E0089583E0089581E007
:103BA0000895982F973068F59093E900981739F0A9
:103BB0007091EC002091ED005091F00003C0242F93
:103BC000762F50E021FD02C09F5FECCF3091EB00DB
:103BD0003E7F3093EB003091ED003D7F3093ED0060
:103BE0003091EB0031603093EB007093EC00209348
:103BF000ED005093F0002091EE0027FDE5CF80E02E
:103C000008958F708093E90081E0089580917B0290
:103C100087FF11C08091E80082FD05C080917A0283
:103C20008111F8CF11C08091E8008B770BC0809193
:103C30007A02882349F08091E80080FFF8CF8091D4
:103C4000E8008E778093E80008952091E400309199
:103C5000E50095E64091EC00842F817040FF23C081
:103C60008091E80080FD1DC080917A02882399F040
:103C7000853099F08091EB0085FD11C04091E40002
:103C80005091E5002417350729F3915011F09A015E
:103C9000E1CF84E0089582E0089583E0089581E013
:103CA000089580E008954091E80042FFDDCF089537
:103CB0000E94C61E0E94CE1EE0EEF0E08081816070
:103CC0008083E8EDF0E080818F77808319BCA7EDD9
:103CD000B0E08C918E7F8C9380818F7E8083109258
:103CE000790208950F931F93CF93DF930E94C61E0E
:103CF0000E94CE1EC8EDD0E088818F7788838881AE
:103D00008068888388818F7D888319BC10927A02AD
:103D100010927602109278021092770200EE10E074
:103D2000F80180818B7F808388818160888342E075
:103D300060E080E00E94D11DE1EEF0E080818E7FA6
:103D40008083E2EEF0E08081816080838081886002
:103D50008083F80180818E7F808388818061888361
:103D6000DF91CF911F910F910895E8EDF0E08081F0
:103D70008F7E8083E7EDF0E080818160808384E046
:103D800082BF81E0809379020C94721EE8EDF0E02E
:103D900080818E7F80831092E20008951092DA0075
:103DA0001092E10008951F920F920FB60F92112406
:103DB0002F933F934F935F936F937F938F939F9333
:103DC000AF93BF93EF93FF938091E10082FF0BC00D
:103DD0008091E20082FF07C08091E1008B7F809399
:103DE000E1000E9449218091DA0080FF1FC080918C
:103DF000D80080FF1BC08091DA008E7F8093DA00AC
:103E00008091D90080FF0DC080E189BD82E189BD2C
:103E100009B400FEFDCF81E080937A020E941B1B53
:103E200005C019BC10927A020E94291B8091E10002
:103E300080FF19C08091E20080FF15C08091E200F0
:103E40008E7F8093E2008091E20080618093E200A7
:103E50008091D80080628093D80019BC85E080935F
:103E60007A020E942E1B8091E10084FF30C0809175
:103E7000E20084FF2CC080E189BD82E189BD09B4E4
:103E800000FEFDCF8091D8008F7D8093D800809177
:103E9000E1008F7E8093E1008091E2008F7E80932D
:103EA000E2008091E20081608093E20080917602DE
:103EB000882311F084E007C08091E30087FD02C0F1
:103EC00081E001C083E080937A020E94361B8091DA
:103ED000E10083FF29C08091E20083FF25C080912B
:103EE000E100877F8093E10082E080937A02109264
:103EF00076028091E1008E7F8093E1008091E20064
:103F00008E7F8093E2008091E20080618093E200E6
:103F100042E060E080E00E94D11D8091F000886066
:103F20008093F0000E942C1BFF91EF91BF91AF9105
:103F30009F918F917F916F915F914F913F912F91C1
:103F40000F900FBE0F901F9018951F920F920FB6F3
:103F50000F9211242F933F934F935F936F937F930F
:103F60008F939F93AF93BF93CF93DF93EF93FF9381
:103F7000C091E900CF708091EC00D82FD17080FD06
:103F8000D0E81092E9008091F000877F8093F000E4
:103F900078940E94E91F1092E9008091F0008860F7
:103FA0008093F000CD2BCF70C093E900FF91EF918B
:103FB000DF91CF91BF91AF919F918F917F916F9141
:103FC0005F914F913F912F910F900FBE0F901F90D7
:103FD00018951F93CF93DF93CDB7DEB7AA970FB68F
:103FE000F894DEBF0FBECDBFEBE7F2E08091F100A9
:103FF000819322E0E338F207C9F70E94541B8091B5
:10400000E80083FF2EC180917B0290917C02492FB2
:1040100050E04A30510508F024C1FA01EF55FF4F36
:104020000C947921803821F0823809F01AC108C037
:104030008091770290917802992389F082600FC075
:1040400080917F028F70873008F00BC18093E90068
:104050008091EB0085FB882780F91092E900909110
:10406000E800977F9093E8008093F1001092F100B0
:10407000D1C0282F2D7F09F0F4C0882319F0823099
:1040800061F0EFC080917D02813009F0EAC0933089
:1040900009F080E0809378022EC080917D0281112A
:1040A0002AC080917F028F702FEF280F263008F0F2
:1040B000D8C08093E9002091EB0020FF1CC0933012
:1040C00021F48091EB00806214C09091EB0090612C
:1040D0009093EB0021E030E0A90102C0440F551F8E
:1040E0008A95E2F74093EA001092EA008091EB0093
:1040F00088608093EB001092E9008091E800877F50
:104100008093E8000E94061EACC08111AAC01091E5
:104110007D021F778091E3008078812B8093E300FC
:104120008091E800877F8093E8000E94061E8091BE
:10413000E80080FFFCCF8091E30080688093E3007B
:10414000111102C082E001C083E080937A0289C02D
:104150008058823008F085C080917D0290917E0267
:104160008C3D53E0950779F583E08A838AE2898361
:104170004FB7F894DE01139620E03EE051E2E32FC2
:10418000F0E050935700E49120FF03C0E295EF70F8
:104190003F5FEF708E2F90E0EA3010F0C79601C0BD
:1041A000C0968D939D932F5F243149F74FBF809127
:1041B000E800877F8093E8006AE270E0CE01019614
:1041C0000E94121D16C060917F0270918002AE01A4
:1041D0004F5F5F4F0E94561CBC01892B09F441C000
:1041E0009091E800977F9093E80089819A810E94DE
:1041F000701D8091E8008B778093E80032C0803892
:1042000081F58091E800877F8093E80080917602B5
:104210008093F1008091E8008E7772CF811121C0E8
:1042200080917D0290917E0299270297D4F480912B
:10423000E800877F8093E80080917D02809376027A
:104240000E94061E80917602811106C08091E300D3
:1042500087FD02C081E001C084E080937A020E9461
:10426000401B8091E80083FF0AC08091E800877FAF
:104270008093E8008091EB0080628093EB00AA9627
:104280000FB6F894DEBF0FBECDBFDF91CF911F9167
:1042900008950895CF9380917A028823A1F0C09168
:1042A000E900CF709091EC00892F817090FD80E83B
:1042B000C82B1092E9008091E80083FD0E94E91F5D
:1042C000CF70C093E900CF91089597FB072E16F4A5
:1042D000009407D077FD09D00E947F2107FC05D00C
:1042E0003EF4909581959F4F0895709561957F4F0D
:1042F0000895EE0FFF1F0590F491E02D0994AA1B7D
:10430000BB1B51E107C0AA1FBB1FA617B70710F0C0
:10431000A61BB70B881F991F5A95A9F780959095F2
:10432000BC01CD010895FB01DC0104C08D91019019
:10433000801921F441505040C8F7881B990B08950B
:10434000F999FECF92BD81BDF89A992780B508955D
:10435000A8E1B0E042E050E00C94D421262FF99976
:10436000FECF92BD81BDF89A019700B4021639F0D4
:104370001FBA20BD0FB6F894FA9AF99A0FBE0895A5
:104380000396272F0E94AF210E94AE21252F0E9465
:10439000AF21242F0C94AF210196272F0E94AF212B
:1043A0000C94AE21DC01CB01FC01F999FECF06C0D3
:1043B000F2BDE1BDF89A319600B40D9241505040E3
:0843C000B8F70895F894FFCF4F
:1043C800C800F401280850011E0A1401841AA71A0B
:1043D800881A171B131B871A01E200E900EA00B5C7
:1043E80000B600B700CD008301CC008A0192019489
:1043F800012102230224022502260227022A02B3EF
:1044080000B4006F007000818283E200E900EA00D6
:10441800B500B600B700CD008301CC008A01920137
:1044280094012102230224022502260227022A02DD
:10443800B300B4006F007000818283F1F49694F0A9
:04444800F5973400B0
:00000001FF
